 sunmscapi

 Timestamp is 44fc4735 (reproducible build file hash)

 Preferred load address is 0000000180000000

 Start         Length     Name                   Class
 0001:00000000 00000020H .text$di                CODE
 0001:00000020 00004fe0H .text$mn                CODE
 0001:00005000 00000036H .text$mn$00             CODE
 0001:00005036 000005f5H .text$x                 CODE
 0002:00000000 00000338H .idata$5                DATA
 0002:00000338 00000038H .00cfg                  DATA
 0002:00000370 00000008H .CRT$XCA                DATA
 0002:00000378 00000008H .CRT$XCU                DATA
 0002:00000380 00000008H .CRT$XCZ                DATA
 0002:00000388 00000008H .CRT$XIA                DATA
 0002:00000390 00000008H .CRT$XIZ                DATA
 0002:00000398 00000008H .CRT$XPA                DATA
 0002:000003a0 00000008H .CRT$XPZ                DATA
 0002:000003a8 00000008H .CRT$XTA                DATA
 0002:000003b0 00000010H .CRT$XTZ                DATA
 0002:000003b8 00000000H .gehcont$y              DATA
 0002:000003b8 00000000H .gfids$y                DATA
 0002:000003c0 00000940H .rdata                  DATA
 0002:00000d00 00000000H .rdata$CastGuardVftablesA DATA
 0002:00000d00 00000000H .rdata$CastGuardVftablesC DATA
 0002:00000d00 000001f4H .rdata$r                DATA
 0002:00000ef4 00000078H .rdata$voltmd           DATA
 0002:00000f6c 00000334H .rdata$zzzdbg           DATA
 0002:000012a0 00000008H .rtc$IAA                DATA
 0002:000012a8 00000008H .rtc$IZZ                DATA
 0002:000012b0 00000008H .rtc$TAA                DATA
 0002:000012b8 00000008H .rtc$TZZ                DATA
 0002:000012c0 00000690H .xdata                  DATA
 0002:00001950 000000f0H .xdata$x                DATA
 0002:00001a40 00000698H .edata                  DATA
 0002:000020d8 000000f0H .idata$2                DATA
 0002:000021c8 00000018H .idata$3                DATA
 0002:000021e0 00000338H .idata$4                DATA
 0002:00002518 00000894H .idata$6                DATA
 0003:00000000 00000078H .data                   DATA
 0003:00000078 00000080H .data$r                 DATA
 0003:000000f8 00000028H .data$rs                DATA
 0003:00000120 00000608H .bss                    DATA
 0004:00000000 00000540H .pdata                  DATA
 0005:00000000 00000060H .rsrc$01                DATA
 0005:00000060 00000320H .rsrc$02                DATA

  Address         Publics by Value              Rva+Base               Lib:Object

 0000:00000000       __AbsoluteZero             0000000000000000     <absolute>
 0000:00000000       ___safe_se_handler_count   0000000000000000     <absolute>
 0000:00000000       ___safe_se_handler_table   0000000000000000     <absolute>
 0000:00000000       __arm64x_extra_rfe_table   0000000000000000     <absolute>
 0000:00000000       __arm64x_extra_rfe_table_size 0000000000000000     <absolute>
 0000:00000000       __arm64x_native_entrypoint 0000000000000000     <absolute>
 0000:00000000       __arm64x_redirection_metadata 0000000000000000     <absolute>
 0000:00000000       __arm64x_redirection_metadata_count 0000000000000000     <absolute>
 0000:00000000       __dynamic_value_reloc_table 0000000000000000     <absolute>
 0000:00000000       __enclave_config           0000000000000000     <absolute>
 0000:00000000       __guard_check_icall_a64n_fptr 0000000000000000     <absolute>
 0000:00000000       __guard_eh_cont_count      0000000000000000     <absolute>
 0000:00000000       __guard_eh_cont_table      0000000000000000     <absolute>
 0000:00000000       __guard_fids_count         0000000000000000     <absolute>
 0000:00000000       __guard_fids_table         0000000000000000     <absolute>
 0000:00000000       __guard_iat_count          0000000000000000     <absolute>
 0000:00000000       __guard_iat_table          0000000000000000     <absolute>
 0000:00000000       __guard_longjmp_count      0000000000000000     <absolute>
 0000:00000000       __guard_longjmp_table      0000000000000000     <absolute>
 0000:00000000       __hybrid_auxiliary_delayload_iat 0000000000000000     <absolute>
 0000:00000000       __hybrid_auxiliary_delayload_iat_copy 0000000000000000     <absolute>
 0000:00000000       __hybrid_auxiliary_iat     0000000000000000     <absolute>
 0000:00000000       __hybrid_auxiliary_iat_copy 0000000000000000     <absolute>
 0000:00000000       __hybrid_code_map          0000000000000000     <absolute>
 0000:00000000       __hybrid_code_map_count    0000000000000000     <absolute>
 0000:00000000       __hybrid_image_info_bitfield 0000000000000000     <absolute>
 0000:00000000       __x64_code_ranges_to_entry_points 0000000000000000     <absolute>
 0000:00000000       __x64_code_ranges_to_entry_points_count 0000000000000000     <absolute>
 0000:00000100       __guard_flags              0000000000000100     <absolute>
 0000:00000000       __ImageBase                0000000180000000     <linker-defined>
 0001:00000020       ?CallStaticObjectMethod@JNIEnv_@@QEAAPEAV_jobject@@PEAV_jclass@@PEAU_jmethodID@@ZZ 0000000180001020 f i security.obj
 0001:00000044       ?CallVoidMethod@JNIEnv_@@QEAAXPEAV_jobject@@PEAU_jmethodID@@ZZ 0000000180001044 f i security.obj
 0001:00000068       ?NewObject@JNIEnv_@@QEAAPEAV_jobject@@PEAV_jclass@@PEAU_jmethodID@@ZZ 0000000180001068 f i security.obj
 0001:0000008c       GetCertificateChain        000000018000108c f   security.obj
 0001:000000f0       Java_sun_security_mscapi_CKeyPairGenerator_00024RSA_generateCKeyPair 00000001800010f0 f   security.obj
 0001:0000026c       Java_sun_security_mscapi_CKeyStore_destroyKeyContainer 000000018000126c f   security.obj
 0001:0000030c       Java_sun_security_mscapi_CKeyStore_generateRSAPrivateKeyBlob 000000018000130c f   security.obj
 0001:00000378       Java_sun_security_mscapi_CKeyStore_loadKeysOrCertificateChains 0000000180001378 f   security.obj
 0001:00000f58       Java_sun_security_mscapi_CKeyStore_removeCertificate 0000000180001f58 f   security.obj
 0001:00001204       Java_sun_security_mscapi_CKeyStore_removeCngKey 0000000180002204 f   security.obj
 0001:00001234       Java_sun_security_mscapi_CKeyStore_storeCertificate 0000000180002234 f   security.obj
 0001:00001790       Java_sun_security_mscapi_CKeyStore_storePrivateKey 0000000180002790 f   security.obj
 0001:00001958       Java_sun_security_mscapi_CKey_cleanUp 0000000180002958 f   security.obj
 0001:00001998       Java_sun_security_mscapi_CKey_getContainerName 0000000180002998 f   security.obj
 0001:00001a10       Java_sun_security_mscapi_CKey_getKeyType 0000000180002a10 f   security.obj
 0001:00001ad0       Java_sun_security_mscapi_CPublicKey_00024CRSAPublicKey_getExponent 0000000180002ad0 f   security.obj
 0001:00001c2c       Java_sun_security_mscapi_CPublicKey_00024CRSAPublicKey_getModulus 0000000180002c2c f   security.obj
 0001:00001dac       Java_sun_security_mscapi_CPublicKey_getPublicKeyBlob 0000000180002dac f   security.obj
 0001:00001f80       Java_sun_security_mscapi_CRSACipher_cngEncryptDecrypt 0000000180002f80 f   security.obj
 0001:00002118       Java_sun_security_mscapi_CRSACipher_encryptDecrypt 0000000180003118 f   security.obj
 0001:0000237c       Java_sun_security_mscapi_CSignature_00024RSA_generatePublicKeyBlob 000000018000337c f   security.obj
 0001:000023bc       Java_sun_security_mscapi_CSignature_importECPublicKey 00000001800033bc f   security.obj
 0001:00002554       Java_sun_security_mscapi_CSignature_importPublicKey 0000000180003554 f   security.obj
 0001:000026e4       Java_sun_security_mscapi_CSignature_signCngHash 00000001800036e4 f   security.obj
 0001:00002a18       Java_sun_security_mscapi_CSignature_signHash 0000000180003a18 f   security.obj
 0001:00002d24       Java_sun_security_mscapi_CSignature_verifyCngSignedHash 0000000180003d24 f   security.obj
 0001:00002fa4       Java_sun_security_mscapi_CSignature_verifySignedHash 0000000180003fa4 f   security.obj
 0001:000031e8       Java_sun_security_mscapi_PRNG_generateSeed 00000001800041e8 f   security.obj
 0001:00003348       Java_sun_security_mscapi_PRNG_getContext 0000000180004348 f   security.obj
 0001:0000339c       Java_sun_security_mscapi_PRNG_releaseContext 000000018000439c f   security.obj
 0001:000033b8       MapHashAlgorithm           00000001800043b8 f   security.obj
 0001:00003500       MapHashIdentifier          0000000180004500 f   security.obj
 0001:000035f4       ThrowException             00000001800045f4 f   security.obj
 0001:000036b8       ThrowExceptionWithMessage  00000001800046b8 f   security.obj
 0001:000036f0       ThrowExceptionWithMessageAndErrcode 00000001800046f0 f   security.obj
 0001:000037c0       __local_stdio_printf_options 00000001800047c0 f i security.obj
 0001:000037c8       convertToLittleEndian      00000001800047c8 f   security.obj
 0001:000038bc       dump                       00000001800048bc f   security.obj
 0001:000039e0       fprintf                    00000001800049e0 f i security.obj
 0001:00003a24       generateKeyBlob            0000000180004a24 f   security.obj
 0001:00003cbc       new[]                      0000000180004cbc f   security.obj
 0001:00003d04       printf                     0000000180004d04 f i security.obj
 0001:00003d58       snprintf                   0000000180004d58 f i security.obj
 0001:00003daf       NCryptOpenStorageProvider  0000000180004daf f   ncrypt:ncrypt.dll
 0001:00003db5       NCryptGetProperty          0000000180004db5 f   ncrypt:ncrypt.dll
 0001:00003dbb       NCryptEncrypt              0000000180004dbb f   ncrypt:ncrypt.dll
 0001:00003dc1       NCryptDecrypt              0000000180004dc1 f   ncrypt:ncrypt.dll
 0001:00003dc7       NCryptImportKey            0000000180004dc7 f   ncrypt:ncrypt.dll
 0001:00003dcd       NCryptExportKey            0000000180004dcd f   ncrypt:ncrypt.dll
 0001:00003dd3       NCryptSignHash             0000000180004dd3 f   ncrypt:ncrypt.dll
 0001:00003dd9       NCryptVerifySignature      0000000180004dd9 f   ncrypt:ncrypt.dll
 0001:00003ddf       NCryptDeleteKey            0000000180004ddf f   ncrypt:ncrypt.dll
 0001:00003de5       NCryptFreeObject           0000000180004de5 f   ncrypt:ncrypt.dll
 0001:00003deb       NCryptTranslateHandle      0000000180004deb f   ncrypt:ncrypt.dll
 0001:00003df4       ??3@YAXPEAX_K@Z            0000000180004df4 f   MSVCRT:delete_scalar_size.obj
 0001:00003df4       ??_V@YAXPEAX@Z             0000000180004df4 f   MSVCRT:delete_array.obj
 0001:00003dfc       ??_U@YAPEAX_KAEBUnothrow_t@std@@@Z 0000000180004dfc f   MSVCRT:new_array_nothrow.obj
 0001:00003e04       __GSHandlerCheck           0000000180004e04 f   MSVCRT:gshandler.obj
 0001:00003e24       __GSHandlerCheckCommon     0000000180004e24 f   MSVCRT:gshandler.obj
 0001:00003e80       __GSHandlerCheck_SEH       0000000180004e80 f   MSVCRT:gshandlerseh.obj
 0001:00003f20       __chkstk                   0000000180004f20 f   MSVCRT:chkstk.obj
 0001:00003f20       _alloca_probe              0000000180004f20 f   MSVCRT:chkstk.obj
 0001:00003f80       __security_check_cookie    0000000180004f80 f   MSVCRT:amdsecgs.obj
 0001:000042b0       _DllMainCRTStartup         00000001800052b0 f   MSVCRT:dll_dllmain.obj
 0001:000042f0       ??3@YAXPEAX@Z              00000001800052f0 f   MSVCRT:delete_scalar.obj
 0001:000042f8       ??2@YAPEAX_KAEBUnothrow_t@std@@@Z 00000001800052f8 f   MSVCRT:new_scalar_nothrow.obj
 0001:0000430c       __raise_securityfailure    000000018000530c f   MSVCRT:gs_report.obj
 0001:00004340       __report_gsfailure         0000000180005340 f   MSVCRT:gs_report.obj
 0001:00004488       __security_init_cookie     0000000180005488 f   MSVCRT:gs_support.obj
 0001:00004534       DllMain                    0000000180005534 f   MSVCRT:dll_dllmain_stub.obj
 0001:00004558       ?__scrt_initialize_type_info@@YAXXZ 0000000180005558 f   MSVCRT:tncleanup.obj
 0001:00004568       ?__scrt_uninitialize_type_info@@YAXXZ 0000000180005568 f   MSVCRT:tncleanup.obj
 0001:00004574       __local_stdio_scanf_options 0000000180005574 f i MSVCRT:default_local_stdio_options.obj
 0001:0000457c       __scrt_initialize_default_local_stdio_options 000000018000557c f   MSVCRT:default_local_stdio_options.obj
 0001:00004598       __scrt_acquire_startup_lock 0000000180005598 f   MSVCRT:utility.obj
 0001:000045d4       __scrt_dllmain_after_initialize_c 00000001800055d4 f   MSVCRT:utility.obj
 0001:00004608       __scrt_dllmain_before_initialize_c 0000000180005608 f   MSVCRT:utility.obj
 0001:00004620       __scrt_dllmain_crt_thread_attach 0000000180005620 f   MSVCRT:utility.obj
 0001:00004648       __scrt_dllmain_crt_thread_detach 0000000180005648 f   MSVCRT:utility.obj
 0001:00004660       __scrt_dllmain_exception_filter 0000000180005660 f   MSVCRT:utility.obj
 0001:000046c0       __scrt_dllmain_uninitialize_c 00000001800056c0 f   MSVCRT:utility.obj
 0001:000046f0       __scrt_dllmain_uninitialize_critical 00000001800056f0 f   MSVCRT:utility.obj
 0001:00004704       __scrt_initialize_crt      0000000180005704 f   MSVCRT:utility.obj
 0001:00004740       __scrt_initialize_onexit_tables 0000000180005740 f   MSVCRT:utility.obj
 0001:000047cc       __scrt_is_nonwritable_in_current_image 00000001800057cc f   MSVCRT:utility.obj
 0001:00004864       __scrt_release_startup_lock 0000000180005864 f   MSVCRT:utility.obj
 0001:00004888       __scrt_uninitialize_crt    0000000180005888 f   MSVCRT:utility.obj
 0001:000048b4       __scrt_get_dyn_tls_init_callback 00000001800058b4 f   MSVCRT:dyn_tls_init.obj
 0001:000048bc       __crt_debugger_hook        00000001800058bc f   MSVCRT:utility_desktop.obj
 0001:000048c4       __scrt_fastfail            00000001800058c4 f   MSVCRT:utility_desktop.obj
 0001:00004a0c       _RTC_Initialize            0000000180005a0c f   MSVCRT:initsect.obj
 0001:00004a48       _RTC_Terminate             0000000180005a48 f   MSVCRT:initsect.obj
 0001:00004a84       _guard_check_icall_nop     0000000180005a84 f i MSVCRT:guard_support.obj
 0001:00004a88       ??2@YAPEAX_K@Z             0000000180005a88 f   MSVCRT:new_scalar.obj
 0001:00004ac4       __isa_available_init       0000000180005ac4 f   MSVCRT:cpu_disp.obj
 0001:00004d90       _get_startup_argv_mode     0000000180005d90 f   MSVCRT:argv_mode.obj
 0001:00004d98       __scrt_is_ucrt_dll_in_use  0000000180005d98 f   MSVCRT:ucrt_detection.obj
 0001:00004db0       ??0bad_alloc@std@@QEAA@AEBV01@@Z 0000000180005db0 f i MSVCRT:throw_bad_alloc.obj
 0001:00004dec       ??0bad_alloc@std@@QEAA@XZ  0000000180005dec f i MSVCRT:throw_bad_alloc.obj
 0001:00004e0c       ??0bad_array_new_length@std@@QEAA@AEBV01@@Z 0000000180005e0c f i MSVCRT:throw_bad_alloc.obj
 0001:00004e48       ??0bad_array_new_length@std@@QEAA@XZ 0000000180005e48 f i MSVCRT:throw_bad_alloc.obj
 0001:00004e68       ??0exception@std@@QEAA@AEBV01@@Z 0000000180005e68 f i MSVCRT:throw_bad_alloc.obj
 0001:00004e9c       ??1bad_alloc@std@@UEAA@XZ  0000000180005e9c f i MSVCRT:throw_bad_alloc.obj
 0001:00004e9c       ??1bad_array_new_length@std@@UEAA@XZ 0000000180005e9c f i MSVCRT:throw_bad_alloc.obj
 0001:00004eb0       ??_Ebad_alloc@std@@UEAAPEAXI@Z 0000000180005eb0 f i MSVCRT:throw_bad_alloc.obj
 0001:00004eb0       ??_Ebad_array_new_length@std@@UEAAPEAXI@Z 0000000180005eb0 f i MSVCRT:throw_bad_alloc.obj
 0001:00004eb0       ??_Eexception@std@@UEAAPEAXI@Z 0000000180005eb0 f i MSVCRT:throw_bad_alloc.obj
 0001:00004eb0       ??_Gbad_alloc@std@@UEAAPEAXI@Z 0000000180005eb0 f i MSVCRT:throw_bad_alloc.obj
 0001:00004eb0       ??_Gbad_array_new_length@std@@UEAAPEAXI@Z 0000000180005eb0 f i MSVCRT:throw_bad_alloc.obj
 0001:00004eb0       ??_Gexception@std@@UEAAPEAXI@Z 0000000180005eb0 f i MSVCRT:throw_bad_alloc.obj
 0001:00004ef4       ?__scrt_throw_std_bad_alloc@@YAXXZ 0000000180005ef4 f   MSVCRT:throw_bad_alloc.obj
 0001:00004f14       ?__scrt_throw_std_bad_array_new_length@@YAXXZ 0000000180005f14 f   MSVCRT:throw_bad_alloc.obj
 0001:00004f34       ?what@exception@std@@UEBAPEBDXZ 0000000180005f34 f i MSVCRT:throw_bad_alloc.obj
 0001:00004f48       ??_Etype_info@@UEAAPEAXI@Z 0000000180005f48 f i MSVCRT:std_type_info_static.obj
 0001:00004f48       ??_Gtype_info@@UEAAPEAXI@Z 0000000180005f48 f i MSVCRT:std_type_info_static.obj
 0001:00004f73       memcpy                     0000000180005f73 f   vcruntime:VCRUNTIME140.dll
 0001:00004f79       memset                     0000000180005f79 f   vcruntime:VCRUNTIME140.dll
 0001:00004f7f       __C_specific_handler       0000000180005f7f f   vcruntime:VCRUNTIME140.dll
 0001:00004f85       _local_unwind              0000000180005f85 f   vcruntime:VCRUNTIME140.dll
 0001:00004f8b       __CxxFrameHandler4         0000000180005f8b f   vcruntime:VCRUNTIME140_1.dll
 0001:00004f91       __std_type_info_destroy_list 0000000180005f91 f   vcruntime:VCRUNTIME140.dll
 0001:00004f97       __std_exception_copy       0000000180005f97 f   vcruntime:VCRUNTIME140.dll
 0001:00004f9d       __std_exception_destroy    0000000180005f9d f   vcruntime:VCRUNTIME140.dll
 0001:00004fa3       _CxxThrowException         0000000180005fa3 f   vcruntime:VCRUNTIME140.dll
 0001:00004fa9       strcmp                     0000000180005fa9 f   ucrt:api-ms-win-crt-string-l1-1-0.dll
 0001:00004faf       strcpy                     0000000180005faf f   ucrt:api-ms-win-crt-string-l1-1-0.dll
 0001:00004fb5       _initterm                  0000000180005fb5 f   ucrt:api-ms-win-crt-runtime-l1-1-0.dll
 0001:00004fbb       _initterm_e                0000000180005fbb f   ucrt:api-ms-win-crt-runtime-l1-1-0.dll
 0001:00004fc1       free                       0000000180005fc1 f   ucrt:api-ms-win-crt-heap-l1-1-0.dll
 0001:00004fc7       _seh_filter_dll            0000000180005fc7 f   ucrt:api-ms-win-crt-runtime-l1-1-0.dll
 0001:00004fcd       _configure_narrow_argv     0000000180005fcd f   ucrt:api-ms-win-crt-runtime-l1-1-0.dll
 0001:00004fd3       _initialize_narrow_environment 0000000180005fd3 f   ucrt:api-ms-win-crt-runtime-l1-1-0.dll
 0001:00004fd9       _initialize_onexit_table   0000000180005fd9 f   ucrt:api-ms-win-crt-runtime-l1-1-0.dll
 0001:00004fdf       _execute_onexit_table      0000000180005fdf f   ucrt:api-ms-win-crt-runtime-l1-1-0.dll
 0001:00004fe5       _cexit                     0000000180005fe5 f   ucrt:api-ms-win-crt-runtime-l1-1-0.dll
 0001:00004feb       _callnewh                  0000000180005feb f   ucrt:api-ms-win-crt-heap-l1-1-0.dll
 0001:00004ff1       malloc                     0000000180005ff1 f   ucrt:api-ms-win-crt-heap-l1-1-0.dll
 0001:00004ff8       __acrt_initialize          0000000180005ff8 f   MSVCRT:ucrt_stubs.obj
 0001:00004ff8       __acrt_thread_attach       0000000180005ff8 f   MSVCRT:ucrt_stubs.obj
 0001:00004ff8       __acrt_thread_detach       0000000180005ff8 f   MSVCRT:ucrt_stubs.obj
 0001:00004ff8       __acrt_uninitialize        0000000180005ff8 f   MSVCRT:ucrt_stubs.obj
 0001:00004ff8       __acrt_uninitialize_critical 0000000180005ff8 f   MSVCRT:ucrt_stubs.obj
 0001:00004ff8       __scrt_stub_for_acrt_initialize 0000000180005ff8 f   MSVCRT:ucrt_stubs.obj
 0001:00004ff8       __scrt_stub_for_acrt_thread_attach 0000000180005ff8 f   MSVCRT:ucrt_stubs.obj
 0001:00004ff8       __scrt_stub_for_acrt_thread_detach 0000000180005ff8 f   MSVCRT:ucrt_stubs.obj
 0001:00004ff8       __scrt_stub_for_acrt_uninitialize 0000000180005ff8 f   MSVCRT:ucrt_stubs.obj
 0001:00004ff8       __scrt_stub_for_acrt_uninitialize_critical 0000000180005ff8 f   MSVCRT:ucrt_stubs.obj
 0001:00004ff8       __vcrt_initialize          0000000180005ff8 f   MSVCRT:ucrt_stubs.obj
 0001:00004ff8       __vcrt_thread_attach       0000000180005ff8 f   MSVCRT:ucrt_stubs.obj
 0001:00004ff8       __vcrt_thread_detach       0000000180005ff8 f   MSVCRT:ucrt_stubs.obj
 0001:00004ff8       __vcrt_uninitialize        0000000180005ff8 f   MSVCRT:ucrt_stubs.obj
 0001:00004ff8       __vcrt_uninitialize_critical 0000000180005ff8 f   MSVCRT:ucrt_stubs.obj
 0001:00004ffc       __scrt_stub_for_is_c_termination_complete 0000000180005ffc f   MSVCRT:ucrt_stubs.obj
 0001:00004ffc       _is_c_termination_complete 0000000180005ffc f   MSVCRT:ucrt_stubs.obj
 0001:00005010       _guard_dispatch_icall_nop  0000000180006010 f   MSVCRT:guard_dispatch.obj
 0001:00005030       _guard_xfg_dispatch_icall_nop 0000000180006030 f   MSVCRT:guard_xfg_dispatch.obj
 0002:00000000       __imp_CryptAcquireContextA 0000000180007000     advapi32:ADVAPI32.dll
 0002:00000008       __imp_CryptReleaseContext  0000000180007008     advapi32:ADVAPI32.dll
 0002:00000010       __imp_CryptGenKey          0000000180007010     advapi32:ADVAPI32.dll
 0002:00000018       __imp_CryptDestroyKey      0000000180007018     advapi32:ADVAPI32.dll
 0002:00000020       __imp_CryptSetKeyParam     0000000180007020     advapi32:ADVAPI32.dll
 0002:00000028       __imp_CryptGetKeyParam     0000000180007028     advapi32:ADVAPI32.dll
 0002:00000030       __imp_CryptSetHashParam    0000000180007030     advapi32:ADVAPI32.dll
 0002:00000038       __imp_CryptGetProvParam    0000000180007038     advapi32:ADVAPI32.dll
 0002:00000040       __imp_CryptGenRandom       0000000180007040     advapi32:ADVAPI32.dll
 0002:00000048       __imp_CryptGetUserKey      0000000180007048     advapi32:ADVAPI32.dll
 0002:00000050       __imp_CryptExportKey       0000000180007050     advapi32:ADVAPI32.dll
 0002:00000058       __imp_CryptImportKey       0000000180007058     advapi32:ADVAPI32.dll
 0002:00000060       __imp_CryptEncrypt         0000000180007060     advapi32:ADVAPI32.dll
 0002:00000068       __imp_CryptDecrypt         0000000180007068     advapi32:ADVAPI32.dll
 0002:00000070       __imp_CryptCreateHash      0000000180007070     advapi32:ADVAPI32.dll
 0002:00000078       __imp_CryptDestroyHash     0000000180007078     advapi32:ADVAPI32.dll
 0002:00000080       __imp_CryptSignHashA       0000000180007080     advapi32:ADVAPI32.dll
 0002:00000088       __imp_CryptVerifySignatureA 0000000180007088     advapi32:ADVAPI32.dll
 0002:00000090       \177ADVAPI32_NULL_THUNK_DATA 0000000180007090     advapi32:ADVAPI32.dll
 0002:00000098       __imp_CertOpenStore        0000000180007098     crypt32:CRYPT32.dll
 0002:000000a0       __imp_CertCloseStore       00000001800070a0     crypt32:CRYPT32.dll
 0002:000000a8       __imp_CertEnumCertificatesInStore 00000001800070a8     crypt32:CRYPT32.dll
 0002:000000b0       __imp_CertFindCertificateInStore 00000001800070b0     crypt32:CRYPT32.dll
 0002:000000b8       __imp_CertCreateCertificateContext 00000001800070b8     crypt32:CRYPT32.dll
 0002:000000c0       __imp_CertFreeCertificateContext 00000001800070c0     crypt32:CRYPT32.dll
 0002:000000c8       __imp_CertSetCertificateContextProperty 00000001800070c8     crypt32:CRYPT32.dll
 0002:000000d0       __imp_CertAddCertificateContextToStore 00000001800070d0     crypt32:CRYPT32.dll
 0002:000000d8       __imp_CertDeleteCertificateFromStore 00000001800070d8     crypt32:CRYPT32.dll
 0002:000000e0       __imp_CertGetPublicKeyLength 00000001800070e0     crypt32:CRYPT32.dll
 0002:000000e8       __imp_CryptAcquireCertificatePrivateKey 00000001800070e8     crypt32:CRYPT32.dll
 0002:000000f0       __imp_CertGetNameStringW   00000001800070f0     crypt32:CRYPT32.dll
 0002:000000f8       __imp_CertOpenSystemStoreA 00000001800070f8     crypt32:CRYPT32.dll
 0002:00000100       __imp_CertGetCertificateChain 0000000180007100     crypt32:CRYPT32.dll
 0002:00000108       __imp_CertFreeCertificateChain 0000000180007108     crypt32:CRYPT32.dll
 0002:00000110       \177CRYPT32_NULL_THUNK_DATA 0000000180007110     crypt32:CRYPT32.dll
 0002:00000118       __imp_IsDebuggerPresent    0000000180007118     kernel32:KERNEL32.dll
 0002:00000120       __imp_InitializeSListHead  0000000180007120     kernel32:KERNEL32.dll
 0002:00000128       __imp_DisableThreadLibraryCalls 0000000180007128     kernel32:KERNEL32.dll
 0002:00000130       __imp_GetSystemTimeAsFileTime 0000000180007130     kernel32:KERNEL32.dll
 0002:00000138       __imp_GetCurrentThreadId   0000000180007138     kernel32:KERNEL32.dll
 0002:00000140       __imp_GetCurrentProcessId  0000000180007140     kernel32:KERNEL32.dll
 0002:00000148       __imp_QueryPerformanceCounter 0000000180007148     kernel32:KERNEL32.dll
 0002:00000150       __imp_IsProcessorFeaturePresent 0000000180007150     kernel32:KERNEL32.dll
 0002:00000158       __imp_TerminateProcess     0000000180007158     kernel32:KERNEL32.dll
 0002:00000160       __imp_GetCurrentProcess    0000000180007160     kernel32:KERNEL32.dll
 0002:00000168       __imp_GetLastError         0000000180007168     kernel32:KERNEL32.dll
 0002:00000170       __imp_FormatMessageA       0000000180007170     kernel32:KERNEL32.dll
 0002:00000178       __imp_RtlCaptureContext    0000000180007178     kernel32:KERNEL32.dll
 0002:00000180       __imp_RtlLookupFunctionEntry 0000000180007180     kernel32:KERNEL32.dll
 0002:00000188       __imp_RtlVirtualUnwind     0000000180007188     kernel32:KERNEL32.dll
 0002:00000190       __imp_UnhandledExceptionFilter 0000000180007190     kernel32:KERNEL32.dll
 0002:00000198       __imp_SetUnhandledExceptionFilter 0000000180007198     kernel32:KERNEL32.dll
 0002:000001a0       \177KERNEL32_NULL_THUNK_DATA 00000001800071a0     kernel32:KERNEL32.dll
 0002:000001a8       __imp__local_unwind        00000001800071a8     vcruntime:VCRUNTIME140.dll
 0002:000001b0       __imp___C_specific_handler 00000001800071b0     vcruntime:VCRUNTIME140.dll
 0002:000001b8       __imp_memset               00000001800071b8     vcruntime:VCRUNTIME140.dll
 0002:000001c0       __imp_memcpy               00000001800071c0     vcruntime:VCRUNTIME140.dll
 0002:000001c8       __imp___std_type_info_destroy_list 00000001800071c8     vcruntime:VCRUNTIME140.dll
 0002:000001d0       __imp___std_exception_copy 00000001800071d0     vcruntime:VCRUNTIME140.dll
 0002:000001d8       __imp___std_exception_destroy 00000001800071d8     vcruntime:VCRUNTIME140.dll
 0002:000001e0       __imp__CxxThrowException   00000001800071e0     vcruntime:VCRUNTIME140.dll
 0002:000001e8       \177VCRUNTIME140_NULL_THUNK_DATA 00000001800071e8     vcruntime:VCRUNTIME140.dll
 0002:000001f0       __imp___CxxFrameHandler4   00000001800071f0     vcruntime:VCRUNTIME140_1.dll
 0002:000001f8       \177VCRUNTIME140_1_NULL_THUNK_DATA 00000001800071f8     vcruntime:VCRUNTIME140_1.dll
 0002:00000200       __imp_mbstowcs             0000000180007200     ucrt:api-ms-win-crt-convert-l1-1-0.dll
 0002:00000208       \177api-ms-win-crt-convert-l1-1-0_NULL_THUNK_DATA 0000000180007208     ucrt:api-ms-win-crt-convert-l1-1-0.dll
 0002:00000210       __imp_getenv               0000000180007210     ucrt:api-ms-win-crt-environment-l1-1-0.dll
 0002:00000218       \177api-ms-win-crt-environment-l1-1-0_NULL_THUNK_DATA 0000000180007218     ucrt:api-ms-win-crt-environment-l1-1-0.dll
 0002:00000220       __imp_free                 0000000180007220     ucrt:api-ms-win-crt-heap-l1-1-0.dll
 0002:00000228       __imp__callnewh            0000000180007228     ucrt:api-ms-win-crt-heap-l1-1-0.dll
 0002:00000230       __imp_malloc               0000000180007230     ucrt:api-ms-win-crt-heap-l1-1-0.dll
 0002:00000238       \177api-ms-win-crt-heap-l1-1-0_NULL_THUNK_DATA 0000000180007238     ucrt:api-ms-win-crt-heap-l1-1-0.dll
 0002:00000240       __imp__execute_onexit_table 0000000180007240     ucrt:api-ms-win-crt-runtime-l1-1-0.dll
 0002:00000248       __imp__cexit               0000000180007248     ucrt:api-ms-win-crt-runtime-l1-1-0.dll
 0002:00000250       __imp__initterm_e          0000000180007250     ucrt:api-ms-win-crt-runtime-l1-1-0.dll
 0002:00000258       __imp__initterm            0000000180007258     ucrt:api-ms-win-crt-runtime-l1-1-0.dll
 0002:00000260       __imp__seh_filter_dll      0000000180007260     ucrt:api-ms-win-crt-runtime-l1-1-0.dll
 0002:00000268       __imp__configure_narrow_argv 0000000180007268     ucrt:api-ms-win-crt-runtime-l1-1-0.dll
 0002:00000270       __imp__initialize_narrow_environment 0000000180007270     ucrt:api-ms-win-crt-runtime-l1-1-0.dll
 0002:00000278       __imp__initialize_onexit_table 0000000180007278     ucrt:api-ms-win-crt-runtime-l1-1-0.dll
 0002:00000280       \177api-ms-win-crt-runtime-l1-1-0_NULL_THUNK_DATA 0000000180007280     ucrt:api-ms-win-crt-runtime-l1-1-0.dll
 0002:00000288       __imp_fflush               0000000180007288     ucrt:api-ms-win-crt-stdio-l1-1-0.dll
 0002:00000290       __imp___acrt_iob_func      0000000180007290     ucrt:api-ms-win-crt-stdio-l1-1-0.dll
 0002:00000298       __imp___stdio_common_vfprintf 0000000180007298     ucrt:api-ms-win-crt-stdio-l1-1-0.dll
 0002:000002a0       __imp___stdio_common_vsprintf 00000001800072a0     ucrt:api-ms-win-crt-stdio-l1-1-0.dll
 0002:000002a8       \177api-ms-win-crt-stdio-l1-1-0_NULL_THUNK_DATA 00000001800072a8     ucrt:api-ms-win-crt-stdio-l1-1-0.dll
 0002:000002b0       __imp_wcslen               00000001800072b0     ucrt:api-ms-win-crt-string-l1-1-0.dll
 0002:000002b8       __imp_wcscmp               00000001800072b8     ucrt:api-ms-win-crt-string-l1-1-0.dll
 0002:000002c0       __imp_strcmp               00000001800072c0     ucrt:api-ms-win-crt-string-l1-1-0.dll
 0002:000002c8       __imp_strcpy               00000001800072c8     ucrt:api-ms-win-crt-string-l1-1-0.dll
 0002:000002d0       \177api-ms-win-crt-string-l1-1-0_NULL_THUNK_DATA 00000001800072d0     ucrt:api-ms-win-crt-string-l1-1-0.dll
 0002:000002d8       __imp_NCryptEncrypt        00000001800072d8     ncrypt:ncrypt.dll
 0002:000002e0       __imp_NCryptDecrypt        00000001800072e0     ncrypt:ncrypt.dll
 0002:000002e8       __imp_NCryptGetProperty    00000001800072e8     ncrypt:ncrypt.dll
 0002:000002f0       __imp_NCryptExportKey      00000001800072f0     ncrypt:ncrypt.dll
 0002:000002f8       __imp_NCryptSignHash       00000001800072f8     ncrypt:ncrypt.dll
 0002:00000300       __imp_NCryptVerifySignature 0000000180007300     ncrypt:ncrypt.dll
 0002:00000308       __imp_NCryptOpenStorageProvider 0000000180007308     ncrypt:ncrypt.dll
 0002:00000310       __imp_NCryptDeleteKey      0000000180007310     ncrypt:ncrypt.dll
 0002:00000318       __imp_NCryptFreeObject     0000000180007318     ncrypt:ncrypt.dll
 0002:00000320       __imp_NCryptImportKey      0000000180007320     ncrypt:ncrypt.dll
 0002:00000328       __imp_NCryptTranslateHandle 0000000180007328     ncrypt:ncrypt.dll
 0002:00000330       \177ncrypt_NULL_THUNK_DATA 0000000180007330     ncrypt:ncrypt.dll
 0002:00000338       __guard_check_icall_fptr   0000000180007338     MSVCRT:guard_support.obj
 0002:00000340       __guard_xfg_check_icall_fptr 0000000180007340     MSVCRT:guard_support.obj
 0002:00000348       __guard_dispatch_icall_fptr 0000000180007348     MSVCRT:guard_support.obj
 0002:00000350       __guard_xfg_dispatch_icall_fptr 0000000180007350     MSVCRT:guard_support.obj
 0002:00000358       __guard_xfg_table_dispatch_icall_fptr 0000000180007358     MSVCRT:guard_support.obj
 0002:00000360       __castguard_check_failure_os_handled_fptr 0000000180007360     MSVCRT:guard_support.obj
 0002:00000368       __guard_memcpy_fptr        0000000180007368     vcruntime:softmemtag.obj
 0002:00000370       __xc_a                     0000000180007370     MSVCRT:initializers.obj
 0002:00000380       __xc_z                     0000000180007380     MSVCRT:initializers.obj
 0002:00000388       __xi_a                     0000000180007388     MSVCRT:initializers.obj
 0002:00000390       __xi_z                     0000000180007390     MSVCRT:initializers.obj
 0002:00000398       __xp_a                     0000000180007398     MSVCRT:initializers.obj
 0002:000003a0       __xp_z                     00000001800073a0     MSVCRT:initializers.obj
 0002:000003a8       __xt_a                     00000001800073a8     MSVCRT:initializers.obj
 0002:000003b0       __xt_z                     00000001800073b0     MSVCRT:initializers.obj
 0002:000003c0       ??_C@_0L@DCABDNEG@CAPI_TRACE@ 00000001800073c0     security.obj
 0002:000003d0       ??_C@_0O@EEFELDNF@?$DN?$DN?$DN?$DN?5?$CFs?5?$DN?$DN?$DN?$DN?6@ 00000001800073d0     security.obj
 0002:000003e0       ??_C@_06LNDOODMG@?$CF04x?3?5@ 00000001800073e0     security.obj
 0002:000003e8       ??_C@_02KNHHEEKP@?5?5@     00000001800073e8     security.obj
 0002:000003ec       ??_C@_05BFHEBJNP@?$CF02X?5@ 00000001800073ec     security.obj
 0002:000003f4       ??_C@_03NDEAONJP@?5?5?5@   00000001800073f4     security.obj
 0002:000003f8       ??_C@_01LFCBOECM@?4@       00000001800073f8     security.obj
 0002:000003fc       ??_C@_02HAOIJKIC@?$CFc@    00000001800073fc     security.obj
 0002:00000400       ??_C@_01EEMJAFIK@?6@       0000000180007400     security.obj
 0002:00000408       ??_C@_0O@NIPGCINC@Unknown?5error@ 0000000180007408     security.obj
 0002:00000418       ??_C@_0BC@KCGCKAP@?$CFs?3?5error?5?$CFlu?0?5?$CFs@ 0000000180007418     security.obj
 0002:00000430       ??_C@_0O@LPHKBBPE@error?5?$CFlu?0?5?$CFs@ 0000000180007430     security.obj
 0002:00000440       ??_C@_0CA@OCDEIOEB@Native?5memory?5allocation?5failed@ 0000000180007440     security.obj
 0002:00000460       ??_C@_0BL@ENCPOIKC@java?1lang?1OutOfMemoryError@ 0000000180007460     security.obj
 0002:0000047c       ??_C@_03JAOICCJD@SHA@      000000018000747c     security.obj
 0002:00000480       ??_C@_04KPMLCNGO@SHA1@     0000000180007480     security.obj
 0002:00000488       ??_C@_05HJMENKNE@SHA?91@   0000000180007488     security.obj
 0002:00000490       ??_C@_08IPMGJMCA@SHA1?$CLMD5@ 0000000180007490     security.obj
 0002:000004a0       ??_C@_07DKFLFLPF@SHA?9256@ 00000001800074a0     security.obj
 0002:000004a8       ??_C@_07LIAJMNEB@SHA?9384@ 00000001800074a8     security.obj
 0002:000004b0       ??_C@_07MEOJAOJE@SHA?9512@ 00000001800074b0     security.obj
 0002:000004b8       ??_C@_03GCGHEHKJ@MD5@      00000001800074b8     security.obj
 0002:000004bc       ??_C@_03CNCGNBGO@MD2@      00000001800074bc     security.obj
 0002:000004c0       ??_C@_19DILNDFJH@?$AAS?$AAH?$AAA?$AA1@ 00000001800074c0     security.obj
 0002:000004d0       ??_C@_1O@HECGKAIN@?$AAS?$AAH?$AAA?$AA2?$AA5?$AA6@ 00000001800074d0     security.obj
 0002:000004e0       ??_C@_1O@KOBLHLEG@?$AAS?$AAH?$AAA?$AA3?$AA8?$AA4@ 00000001800074e0     security.obj
 0002:000004f0       ??_C@_1O@GKBAHMNF@?$AAS?$AAH?$AAA?$AA5?$AA1?$AA2@ 00000001800074f0     security.obj
 0002:00000500       ??_C@_0CA@ODKEJAIA@java?1security?1ProviderException@ 0000000180007500     security.obj
 0002:00000520       ??_C@_0P@LDACLLBM@MSCAPI?5?$CI?$CFld?$CJ?3?5@ 0000000180007520     security.obj
 0002:00000530       ??_C@_0CI@LDLDJJPI@jCertStoreLocation?5is?5not?5a?5val@ 0000000180007530     security.obj
 0002:00000558       ??_C@_0CA@MACLKLAA@java?1security?1KeyStoreException@ 0000000180007558     security.obj
 0002:00000578       ??_C@_0BE@GPOIDJOH@java?1util?1ArrayList@ 0000000180007578     security.obj
 0002:0000058c       ??_C@_03GAEACAIP@?$CI?$CJV@ 000000018000758c     security.obj
 0002:00000590       ??_C@_06FALKBLGB@?$DMinit?$DO@ 0000000180007590     security.obj
 0002:00000598       ??_C@_0BM@MIKFLICJ@?$CI?$FLBLjava?1util?1Collection?$DL?$CJV@ 0000000180007598     security.obj
 0002:000005b8       ??_C@_0BE@HGBDNPAN@generateCertificate@ 00000001800075b8     security.obj
 0002:000005d0       ??_C@_0CM@JPBKDHED@?$CILjava?1lang?1String?$DLLjava?1util?1C@ 00000001800075d0     security.obj
 0002:00000600       ??_C@_0BJ@POMOMMIJ@generateCertificateChain@ 0000000180007600     security.obj
 0002:00000620       ??_C@_0DA@FHNPPNIC@?$CIZLjava?1lang?1String?$DLJJILjava?1ut@ 0000000180007620     security.obj
 0002:00000650       ??_C@_0BP@KJIOGBOH@generateKeyAndCertificateChain@ 0000000180007650     security.obj
 0002:00000670       ??_C@_0BL@JMBEPNBE@?9?9?9?9?9?9?9?9?9?9?9?9?9?9?9?9?9?9?9?9?9?9?9?9?9?9@ 0000000180007670     security.obj
 0002:00000690       ??_C@_0BJ@LOMAEPIP@bHasNoPrivateKey?5?$DN?5TRUE?$CB@ 0000000180007690     security.obj
 0002:000006b0       ??_C@_0BK@PBCGELBN@bHasNoPrivateKey?5?$DN?5TRUE?$CB?$CB@ 00000001800076b0     security.obj
 0002:000006d0       ??_C@_09GGHMOLPI@CNG?5?$CFI64d@ 00000001800076d0     security.obj
 0002:000006e0       ??_C@_0BB@DPFIGFPO@CAPI?5?$CFI64d?5?$CFI64d@ 00000001800076e0     security.obj
 0002:000006f8       ??_C@_0M@MNGGKKAH@2?45?429?437?40@ 00000001800076f8     security.obj
 0002:00000704       ??_C@_06EDLONME@?$CFS?3?5?$CFs@ 0000000180007704     security.obj
 0002:00000710       ??_C@_1BO@LONLFJGG@?$AAA?$AAl?$AAg?$AAo?$AAr?$AAi?$AAt?$AAh?$AAm?$AA?5?$AAN?$AAa?$AAm?$AAe@ 0000000180007710     security.obj
 0002:00000730       ??_C@_0CC@FLCGHJKD@Unknown?5NCRYPT_ALGORITHM_PROPER@ 0000000180007730     security.obj
 0002:00000758       ??_C@_0BO@PMPHIPKH@GetCertificateChain?5failed?5?$CFd@ 0000000180007758     security.obj
 0002:00000778       ??_C@_0CB@OJNKLEOL@java?1security?1SignatureExceptio@ 0000000180007778     security.obj
 0002:000007a0       ??_C@_0BM@BFBFCGA@Unrecognised?5hash?5algorithm@ 00000001800077a0     security.obj
 0002:000007c0       ??_C@_1BM@HFKJNGID@?$AAE?$AAC?$AAC?$AAP?$AAU?$AAB?$AAL?$AAI?$AAC?$AAB?$AAL?$AAO?$AAB@ 00000001800077c0     security.obj
 0002:000007e0       ??_C@_0BL@LLOKBKPE@java?1security?1KeyException@ 00000001800077e0     security.obj
 0002:00000800       ??_C@_0BN@LEDKEDGO@sun?1security?1mscapi?1CKeyPair@ 0000000180007800     security.obj
 0002:00000820       ??_C@_0BJ@HAHEHOOK@?$CILjava?1lang?1String?$DLJJI?$CJV@ 0000000180007820     security.obj
 0002:00000840       ??_C@_09GDNFOKKF@Signature@ 0000000180007840     security.obj
 0002:00000850       ??_C@_08IGAGGAPJ@Exchange@ 0000000180007850     security.obj
 0002:0000085c       ??_C@_03FKNCMABI@?$CFlu@   000000018000785c     security.obj
 0002:00000860       ??_C@_09MGFHLAFE@?$DMUnknown?$DO@ 0000000180007860     security.obj
 0002:00000870       ??_C@_0CP@KCIKFHJG@java?1security?1cert?1CertificateP@ 0000000180007870     security.obj
 0002:000008a0       ??_C@_0BM@PFEPDIKJ@CryptAcquireContext?5failure@ 00000001800078a0     security.obj
 0002:000008c0       ??_C@_0N@GEJMMFOA@Invalid?5BLOB@ 00000001800078c0     security.obj
 0002:000008d0       ??_C@_0BD@GEIFFJNC@Invalid?5key?5length@ 00000001800078d0     security.obj
 0002:000008e8       ??_C@_0CC@LJIPPJAJ@java?1security?1InvalidKeyExcepti@ 00000001800078e8     security.obj
 0002:00000910       ??_C@_0CA@BFBBJNML@sun?1security?1mscapi?1CPrivateKey@ 0000000180007910     security.obj
 0002:00000930       ??_C@_0DJ@LBOEDAIF@?$CILjava?1lang?1String?$DLJJI?$CJLsun?1sec@ 0000000180007930     security.obj
 0002:0000096c       ??_C@_02HAJCGGNB@of@       000000018000796c     security.obj
 0002:00000970       ??_C@_0BA@DCIOBNHG@NCryptImportKey@ 0000000180007970     security.obj
 0002:00000980       ??_C@_1FA@OAAKELHB@?$AAM?$AAi?$AAc?$AAr?$AAo?$AAs?$AAo?$AAf?$AAt?$AA?5?$AAS?$AAo?$AAf?$AAt?$AAw@ 0000000180007980     security.obj
 0002:000009d0       ??_C@_0BP@LCBGNOJP@sun?1security?1mscapi?1CPublicKey@ 00000001800079d0     security.obj
 0002:000009f0       ??_C@_0DI@BHHDKCOH@?$CILjava?1lang?1String?$DLJJI?$CJLsun?1sec@ 00000001800079f0     security.obj
 0002:00000a28       ?nothrow@std@@3Unothrow_t@1@B 0000000180007a28     msvcprt:nothrow.obj
 0002:00000a30       _pDefaultRawDllMain        0000000180007a30     MSVCRT:dll_dllmain.obj
 0002:00000a30       _pRawDllMain               0000000180007a30     MSVCRT:dll_dllmain.obj
 0002:00000a50       __xmm@ffffffffffffffffffffffffffffffff 0000000180007a50     MSVCRT:utility.obj
 0002:00000a68       ??_7exception@std@@6B@     0000000180007a68     MSVCRT:throw_bad_alloc.obj
 0002:00000a78       ??_C@_0BC@EOODALEL@Unknown?5exception@ 0000000180007a78     MSVCRT:throw_bad_alloc.obj
 0002:00000a98       ??_7bad_alloc@std@@6B@     0000000180007a98     MSVCRT:throw_bad_alloc.obj
 0002:00000aa8       ??_C@_0P@GHFPNOJB@bad?5allocation@ 0000000180007aa8     MSVCRT:throw_bad_alloc.obj
 0002:00000ac0       ??_7bad_array_new_length@std@@6B@ 0000000180007ac0     MSVCRT:throw_bad_alloc.obj
 0002:00000ad0       ??_C@_0BF@KINCDENJ@bad?5array?5new?5length@ 0000000180007ad0     MSVCRT:throw_bad_alloc.obj
 0002:00000af0       ??_7type_info@@6B@         0000000180007af0     MSVCRT:std_type_info_static.obj
 0002:00000b00       _load_config_used          0000000180007b00     MSVCRT:loadcfg.obj
 0002:00000d00       ??_R4exception@std@@6B@    0000000180007d00     MSVCRT:throw_bad_alloc.obj
 0002:00000d28       ??_R3exception@std@@8      0000000180007d28     MSVCRT:throw_bad_alloc.obj
 0002:00000d40       ??_R2exception@std@@8      0000000180007d40     MSVCRT:throw_bad_alloc.obj
 0002:00000d50       ??_R1A@?0A@EA@exception@std@@8 0000000180007d50     MSVCRT:throw_bad_alloc.obj
 0002:00000d78       ??_R4bad_array_new_length@std@@6B@ 0000000180007d78     MSVCRT:throw_bad_alloc.obj
 0002:00000da0       ??_R3bad_array_new_length@std@@8 0000000180007da0     MSVCRT:throw_bad_alloc.obj
 0002:00000db8       ??_R2bad_array_new_length@std@@8 0000000180007db8     MSVCRT:throw_bad_alloc.obj
 0002:00000dd8       ??_R1A@?0A@EA@bad_array_new_length@std@@8 0000000180007dd8     MSVCRT:throw_bad_alloc.obj
 0002:00000e00       ??_R1A@?0A@EA@bad_alloc@std@@8 0000000180007e00     MSVCRT:throw_bad_alloc.obj
 0002:00000e28       ??_R3bad_alloc@std@@8      0000000180007e28     MSVCRT:throw_bad_alloc.obj
 0002:00000e40       ??_R2bad_alloc@std@@8      0000000180007e40     MSVCRT:throw_bad_alloc.obj
 0002:00000e58       ??_R4bad_alloc@std@@6B@    0000000180007e58     MSVCRT:throw_bad_alloc.obj
 0002:00000e80       ??_R4type_info@@6B@        0000000180007e80     MSVCRT:std_type_info_static.obj
 0002:00000ea8       ??_R3type_info@@8          0000000180007ea8     MSVCRT:std_type_info_static.obj
 0002:00000ec0       ??_R2type_info@@8          0000000180007ec0     MSVCRT:std_type_info_static.obj
 0002:00000ed0       ??_R1A@?0A@EA@type_info@@8 0000000180007ed0     MSVCRT:std_type_info_static.obj
 0002:00000ef4       __volatile_metadata        0000000180007ef4     <linker-defined>
 0002:000012a0       __rtc_iaa                  00000001800082a0     MSVCRT:initsect.obj
 0002:000012a8       __rtc_izz                  00000001800082a8     MSVCRT:initsect.obj
 0002:000012b0       __rtc_taa                  00000001800082b0     MSVCRT:initsect.obj
 0002:000012b8       __rtc_tzz                  00000001800082b8     MSVCRT:initsect.obj
 0002:00001950       _TI2?AVbad_alloc@std@@     0000000180008950     MSVCRT:throw_bad_alloc.obj
 0002:00001970       _CTA2?AVbad_alloc@std@@    0000000180008970     MSVCRT:throw_bad_alloc.obj
 0002:00001988       _CT??_R0?AVbad_alloc@std@@@8??0bad_alloc@std@@QEAA@AEBV01@@Z24 0000000180008988     MSVCRT:throw_bad_alloc.obj
 0002:000019b0       _CT??_R0?AVexception@std@@@8??0exception@std@@QEAA@AEBV01@@Z24 00000001800089b0     MSVCRT:throw_bad_alloc.obj
 0002:000019d8       _TI3?AVbad_array_new_length@std@@ 00000001800089d8     MSVCRT:throw_bad_alloc.obj
 0002:000019f8       _CTA3?AVbad_array_new_length@std@@ 00000001800089f8     MSVCRT:throw_bad_alloc.obj
 0002:00001a18       _CT??_R0?AVbad_array_new_length@std@@@8??0bad_array_new_length@std@@QEAA@AEBV01@@Z24 0000000180008a18     MSVCRT:throw_bad_alloc.obj
 0002:000020d8       __IMPORT_DESCRIPTOR_ADVAPI32 00000001800090d8     advapi32:ADVAPI32.dll
 0002:000020ec       __IMPORT_DESCRIPTOR_CRYPT32 00000001800090ec     crypt32:CRYPT32.dll
 0002:00002100       __IMPORT_DESCRIPTOR_ncrypt 0000000180009100     ncrypt:ncrypt.dll
 0002:00002114       __IMPORT_DESCRIPTOR_KERNEL32 0000000180009114     kernel32:KERNEL32.dll
 0002:00002128       __IMPORT_DESCRIPTOR_VCRUNTIME140 0000000180009128     vcruntime:VCRUNTIME140.dll
 0002:0000213c       __IMPORT_DESCRIPTOR_VCRUNTIME140_1 000000018000913c     vcruntime:VCRUNTIME140_1.dll
 0002:00002150       __IMPORT_DESCRIPTOR_api-ms-win-crt-stdio-l1-1-0 0000000180009150     ucrt:api-ms-win-crt-stdio-l1-1-0.dll
 0002:00002164       __IMPORT_DESCRIPTOR_api-ms-win-crt-convert-l1-1-0 0000000180009164     ucrt:api-ms-win-crt-convert-l1-1-0.dll
 0002:00002178       __IMPORT_DESCRIPTOR_api-ms-win-crt-environment-l1-1-0 0000000180009178     ucrt:api-ms-win-crt-environment-l1-1-0.dll
 0002:0000218c       __IMPORT_DESCRIPTOR_api-ms-win-crt-string-l1-1-0 000000018000918c     ucrt:api-ms-win-crt-string-l1-1-0.dll
 0002:000021a0       __IMPORT_DESCRIPTOR_api-ms-win-crt-runtime-l1-1-0 00000001800091a0     ucrt:api-ms-win-crt-runtime-l1-1-0.dll
 0002:000021b4       __IMPORT_DESCRIPTOR_api-ms-win-crt-heap-l1-1-0 00000001800091b4     ucrt:api-ms-win-crt-heap-l1-1-0.dll
 0002:000021c8       __NULL_IMPORT_DESCRIPTOR   00000001800091c8     advapi32:ADVAPI32.dll
 0003:00000000       __security_cookie          000000018000a000     MSVCRT:gs_cookie.obj
 0003:00000040       __security_cookie_complement 000000018000a040     MSVCRT:gs_cookie.obj
 0003:00000048       __scrt_native_dllmain_reason 000000018000a048     MSVCRT:utility.obj
 0003:00000050       __isa_inverted             000000018000a050     MSVCRT:cpu_disp.obj
 0003:00000058       __isa_available            000000018000a058     MSVCRT:cpu_disp.obj
 0003:0000005c       __isa_enabled              000000018000a05c     MSVCRT:cpu_disp.obj
 0003:00000060       __memset_fast_string_threshold 000000018000a060     MSVCRT:cpu_disp.obj
 0003:00000068       __memset_nt_threshold      000000018000a068     MSVCRT:cpu_disp.obj
 0003:00000070       __scrt_ucrt_dll_is_in_use  000000018000a070     MSVCRT:ucrt_stubs.obj
 0003:00000078       ??_R0?AVbad_alloc@std@@@8  000000018000a078     MSVCRT:throw_bad_alloc.obj
 0003:000000a0       ??_R0?AVexception@std@@@8  000000018000a0a0     MSVCRT:throw_bad_alloc.obj
 0003:000000c8       ??_R0?AVbad_array_new_length@std@@@8 000000018000a0c8     MSVCRT:throw_bad_alloc.obj
 0003:000000f8       ??_R0?AVtype_info@@@8      000000018000a0f8     MSVCRT:std_type_info_static.obj
 0003:00000120       ?_OptionsStorage@?1??__local_stdio_printf_options@@9@4_KA 000000018000a120     security.obj
 0003:00000128       trace                      000000018000a128     security.obj
 0003:000006b0       ?__type_info_root_node@@3U__type_info_node@@A 000000018000a6b0     MSVCRT:tncleanup.obj
 0003:000006c0       ?_OptionsStorage@?1??__local_stdio_scanf_options@@9@4_KA 000000018000a6c0     MSVCRT:default_local_stdio_options.obj
 0003:000006c8       __scrt_current_native_startup_state 000000018000a6c8     MSVCRT:utility.obj
 0003:000006d0       __scrt_native_startup_lock 000000018000a6d0     MSVCRT:utility.obj
 0003:00000710       __scrt_debugger_hook_flag  000000018000a710     MSVCRT:utility_desktop.obj
 0003:00000714       __avx10_version            000000018000a714     MSVCRT:cpu_disp.obj
 0003:00000718       __favor                    000000018000a718     MSVCRT:cpu_disp.obj
 0003:00000720       __dyn_tls_init_callback    000000018000a720     <common>

 entry point at        0001:000042b0

 Static symbols

 0000:ffff2000       .debug$S                   0000000180000000     sunmscapi.exp
 0000:ffff2000       .debug$S                   0000000180000000     vcruntime:VCRUNTIME140.dll
 0000:ffff2000       .debug$S                   0000000180000000     vcruntime:VCRUNTIME140.dll
 0000:ffff2000       .debug$S                   0000000180000000     vcruntime:VCRUNTIME140.dll
 0000:ffff2000       .debug$S                   0000000180000000     vcruntime:VCRUNTIME140.dll
 0000:ffff2000       .debug$S                   0000000180000000     vcruntime:VCRUNTIME140.dll
 0000:ffff2000       .debug$S                   0000000180000000     vcruntime:VCRUNTIME140.dll
 0000:ffff2000       .debug$S                   0000000180000000     vcruntime:VCRUNTIME140.dll
 0000:ffff2000       .debug$S                   0000000180000000     vcruntime:VCRUNTIME140.dll
 0000:ffff2000       .debug$S                   0000000180000000     vcruntime:VCRUNTIME140.dll
 0000:ffff2000       .debug$S                   0000000180000000     vcruntime:VCRUNTIME140.dll
 0000:ffff2000       .debug$S                   0000000180000000     vcruntime:VCRUNTIME140_1.dll
 0000:ffff2000       .debug$S                   0000000180000000     ucrt:api-ms-win-crt-convert-l1-1-0.dll
 0000:ffff2000       .debug$S                   0000000180000000     ucrt:api-ms-win-crt-environment-l1-1-0.dll
 0000:ffff2000       .debug$S                   0000000180000000     ucrt:api-ms-win-crt-heap-l1-1-0.dll
 0000:ffff2000       .debug$S                   0000000180000000     ucrt:api-ms-win-crt-heap-l1-1-0.dll
 0000:ffff2000       .debug$S                   0000000180000000     ucrt:api-ms-win-crt-heap-l1-1-0.dll
 0000:ffff2000       .debug$S                   0000000180000000     ucrt:api-ms-win-crt-runtime-l1-1-0.dll
 0000:ffff2000       .debug$S                   0000000180000000     ucrt:api-ms-win-crt-runtime-l1-1-0.dll
 0000:ffff2000       .debug$S                   0000000180000000     ucrt:api-ms-win-crt-runtime-l1-1-0.dll
 0000:ffff2000       .debug$S                   0000000180000000     ucrt:api-ms-win-crt-runtime-l1-1-0.dll
 0000:ffff2000       .debug$S                   0000000180000000     ucrt:api-ms-win-crt-runtime-l1-1-0.dll
 0000:ffff2000       .debug$S                   0000000180000000     ucrt:api-ms-win-crt-runtime-l1-1-0.dll
 0000:ffff2000       .debug$S                   0000000180000000     ucrt:api-ms-win-crt-runtime-l1-1-0.dll
 0000:ffff2000       .debug$S                   0000000180000000     ucrt:api-ms-win-crt-runtime-l1-1-0.dll
 0000:ffff2000       .debug$S                   0000000180000000     ucrt:api-ms-win-crt-runtime-l1-1-0.dll
 0000:ffff2000       .debug$S                   0000000180000000     ucrt:api-ms-win-crt-runtime-l1-1-0.dll
 0000:ffff2000       .debug$S                   0000000180000000     ucrt:api-ms-win-crt-runtime-l1-1-0.dll
 0000:ffff2000       .debug$S                   0000000180000000     ucrt:api-ms-win-crt-runtime-l1-1-0.dll
 0000:ffff2000       .debug$S                   0000000180000000     ucrt:api-ms-win-crt-stdio-l1-1-0.dll
 0000:ffff2000       .debug$S                   0000000180000000     ucrt:api-ms-win-crt-stdio-l1-1-0.dll
 0000:ffff2000       .debug$S                   0000000180000000     ucrt:api-ms-win-crt-stdio-l1-1-0.dll
 0000:ffff2000       .debug$S                   0000000180000000     ucrt:api-ms-win-crt-stdio-l1-1-0.dll
 0000:ffff2000       .debug$S                   0000000180000000     ucrt:api-ms-win-crt-string-l1-1-0.dll
 0000:ffff2000       .debug$S                   0000000180000000     ucrt:api-ms-win-crt-string-l1-1-0.dll
 0000:ffff2000       .debug$S                   0000000180000000     ucrt:api-ms-win-crt-string-l1-1-0.dll
 0000:ffff2000       .debug$S                   0000000180000000     ucrt:api-ms-win-crt-string-l1-1-0.dll
 0000:ffff2000       .debug$S                   0000000180000000     advapi32:ADVAPI32.dll
 0000:ffff2000       .debug$S                   0000000180000000     advapi32:ADVAPI32.dll
 0000:ffff2000       .debug$S                   0000000180000000     advapi32:ADVAPI32.dll
 0000:ffff2000       .debug$S                   0000000180000000     advapi32:ADVAPI32.dll
 0000:ffff2000       .debug$S                   0000000180000000     advapi32:ADVAPI32.dll
 0000:ffff2000       .debug$S                   0000000180000000     advapi32:ADVAPI32.dll
 0000:ffff2000       .debug$S                   0000000180000000     advapi32:ADVAPI32.dll
 0000:ffff2000       .debug$S                   0000000180000000     advapi32:ADVAPI32.dll
 0000:ffff2000       .debug$S                   0000000180000000     advapi32:ADVAPI32.dll
 0000:ffff2000       .debug$S                   0000000180000000     advapi32:ADVAPI32.dll
 0000:ffff2000       .debug$S                   0000000180000000     advapi32:ADVAPI32.dll
 0000:ffff2000       .debug$S                   0000000180000000     advapi32:ADVAPI32.dll
 0000:ffff2000       .debug$S                   0000000180000000     advapi32:ADVAPI32.dll
 0000:ffff2000       .debug$S                   0000000180000000     advapi32:ADVAPI32.dll
 0000:ffff2000       .debug$S                   0000000180000000     advapi32:ADVAPI32.dll
 0000:ffff2000       .debug$S                   0000000180000000     advapi32:ADVAPI32.dll
 0000:ffff2000       .debug$S                   0000000180000000     advapi32:ADVAPI32.dll
 0000:ffff2000       .debug$S                   0000000180000000     advapi32:ADVAPI32.dll
 0000:ffff2000       .debug$S                   0000000180000000     crypt32:CRYPT32.dll
 0000:ffff2000       .debug$S                   0000000180000000     crypt32:CRYPT32.dll
 0000:ffff2000       .debug$S                   0000000180000000     crypt32:CRYPT32.dll
 0000:ffff2000       .debug$S                   0000000180000000     crypt32:CRYPT32.dll
 0000:ffff2000       .debug$S                   0000000180000000     crypt32:CRYPT32.dll
 0000:ffff2000       .debug$S                   0000000180000000     crypt32:CRYPT32.dll
 0000:ffff2000       .debug$S                   0000000180000000     crypt32:CRYPT32.dll
 0000:ffff2000       .debug$S                   0000000180000000     crypt32:CRYPT32.dll
 0000:ffff2000       .debug$S                   0000000180000000     crypt32:CRYPT32.dll
 0000:ffff2000       .debug$S                   0000000180000000     crypt32:CRYPT32.dll
 0000:ffff2000       .debug$S                   0000000180000000     crypt32:CRYPT32.dll
 0000:ffff2000       .debug$S                   0000000180000000     crypt32:CRYPT32.dll
 0000:ffff2000       .debug$S                   0000000180000000     crypt32:CRYPT32.dll
 0000:ffff2000       .debug$S                   0000000180000000     crypt32:CRYPT32.dll
 0000:ffff2000       .debug$S                   0000000180000000     crypt32:CRYPT32.dll
 0000:ffff2000       .debug$S                   0000000180000000     kernel32:KERNEL32.dll
 0000:ffff2000       .debug$S                   0000000180000000     kernel32:KERNEL32.dll
 0000:ffff2000       .debug$S                   0000000180000000     kernel32:KERNEL32.dll
 0000:ffff2000       .debug$S                   0000000180000000     kernel32:KERNEL32.dll
 0000:ffff2000       .debug$S                   0000000180000000     kernel32:KERNEL32.dll
 0000:ffff2000       .debug$S                   0000000180000000     kernel32:KERNEL32.dll
 0000:ffff2000       .debug$S                   0000000180000000     kernel32:KERNEL32.dll
 0000:ffff2000       .debug$S                   0000000180000000     kernel32:KERNEL32.dll
 0000:ffff2000       .debug$S                   0000000180000000     kernel32:KERNEL32.dll
 0000:ffff2000       .debug$S                   0000000180000000     kernel32:KERNEL32.dll
 0000:ffff2000       .debug$S                   0000000180000000     kernel32:KERNEL32.dll
 0000:ffff2000       .debug$S                   0000000180000000     kernel32:KERNEL32.dll
 0000:ffff2000       .debug$S                   0000000180000000     kernel32:KERNEL32.dll
 0000:ffff2000       .debug$S                   0000000180000000     kernel32:KERNEL32.dll
 0000:ffff2000       .debug$S                   0000000180000000     kernel32:KERNEL32.dll
 0000:ffff2000       .debug$S                   0000000180000000     kernel32:KERNEL32.dll
 0000:ffff2000       .debug$S                   0000000180000000     kernel32:KERNEL32.dll
 0000:ffff2000       .debug$S                   0000000180000000     kernel32:KERNEL32.dll
 0000:ffff2000       .debug$S                   0000000180000000     kernel32:KERNEL32.dll
 0000:ffff2000       .debug$S                   0000000180000000     ncrypt:ncrypt.dll
 0000:ffff2000       .debug$S                   0000000180000000     ncrypt:ncrypt.dll
 0000:ffff2000       .debug$S                   0000000180000000     ncrypt:ncrypt.dll
 0000:ffff2000       .debug$S                   0000000180000000     ncrypt:ncrypt.dll
 0000:ffff2000       .debug$S                   0000000180000000     ncrypt:ncrypt.dll
 0000:ffff2000       .debug$S                   0000000180000000     ncrypt:ncrypt.dll
 0000:ffff2000       .debug$S                   0000000180000000     ncrypt:ncrypt.dll
 0000:ffff2000       .debug$S                   0000000180000000     ncrypt:ncrypt.dll
 0000:ffff2000       .debug$S                   0000000180000000     ncrypt:ncrypt.dll
 0000:ffff2000       .debug$S                   0000000180000000     ncrypt:ncrypt.dll
 0000:ffff2000       .debug$S                   0000000180000000     ncrypt:ncrypt.dll
 0001:00000000       ??__Etrace@@YAXXZ          0000000180001000 f   security.obj
 0001:00003f10       $$000000                   0000000180004f10     MSVCRT:chkstk.obj
 0001:00003f70       $$000000                   0000000180004f70     MSVCRT:amdsecgs.obj
 0001:00003fa0       ?dllmain_crt_dispatch@@YAHQEAUHINSTANCE__@@KQEAX@Z 0000000180004fa0 f   MSVCRT:dll_dllmain.obj
 0001:00003ff0       ?dllmain_crt_process_attach@@YAHQEAUHINSTANCE__@@QEAX@Z 0000000180004ff0 f   MSVCRT:dll_dllmain.obj
 0001:00004108       ?dllmain_crt_process_detach@@YAH_N@Z 0000000180005108 f   MSVCRT:dll_dllmain.obj
 0001:00004188       ?dllmain_dispatch@@YAHQEAUHINSTANCE__@@KQEAX@Z 0000000180005188 f   MSVCRT:dll_dllmain.obj
 0001:00004414       capture_previous_context   0000000180005414 f   MSVCRT:gs_report.obj
 0001:00005000       $$000000                   0000000180006000     MSVCRT:guard_dispatch.obj
 0001:00005020       $$000000                   0000000180006020     MSVCRT:guard_xfg_dispatch.obj
 0001:00005036       Java_sun_security_mscapi_CKeyPairGenerator_00024RSA_generateCKeyPair$fin$0 0000000180006036 f   security.obj
 0001:00005067       Java_sun_security_mscapi_CKeyStore_destroyKeyContainer$fin$0 0000000180006067 f   security.obj
 0001:00005092       Java_sun_security_mscapi_CKeyStore_loadKeysOrCertificateChains$fin$0 0000000180006092 f   security.obj
 0001:000050ea       Java_sun_security_mscapi_CKeyStore_removeCertificate$fin$0 00000001800060ea f   security.obj
 0001:00005192       Java_sun_security_mscapi_CKeyStore_storeCertificate$fin$0 0000000180006192 f   security.obj
 0001:00005242       Java_sun_security_mscapi_CKeyStore_storePrivateKey$fin$0 0000000180006242 f   security.obj
 0001:0000529a       Java_sun_security_mscapi_CPublicKey_00024CRSAPublicKey_getExponent$fin$0 000000018000629a f   security.obj
 0001:000052dd       Java_sun_security_mscapi_CPublicKey_00024CRSAPublicKey_getModulus$fin$0 00000001800062dd f   security.obj
 0001:00005323       Java_sun_security_mscapi_CPublicKey_getPublicKeyBlob$fin$0 0000000180006323 f   security.obj
 0001:00005323       Java_sun_security_mscapi_CRSACipher_cngEncryptDecrypt$fin$0 0000000180006323 f   security.obj
 0001:00005342       Java_sun_security_mscapi_CRSACipher_encryptDecrypt$fin$0 0000000180006342 f   security.obj
 0001:00005361       Java_sun_security_mscapi_CSignature_importECPublicKey$fin$0 0000000180006361 f   security.obj
 0001:00005371       Java_sun_security_mscapi_CSignature_importPublicKey$fin$0 0000000180006371 f   security.obj
 0001:000053a8       Java_sun_security_mscapi_CSignature_signCngHash$fin$0 00000001800063a8 f   security.obj
 0001:000053ef       Java_sun_security_mscapi_CSignature_signHash$fin$0 00000001800063ef f   security.obj
 0001:0000543f       Java_sun_security_mscapi_CSignature_verifyCngSignedHash$fin$0 000000018000643f f   security.obj
 0001:00005486       Java_sun_security_mscapi_CSignature_verifySignedHash$fin$0 0000000180006486 f   security.obj
 0001:000054d6       Java_sun_security_mscapi_PRNG_generateSeed$fin$0 00000001800064d6 f   security.obj
 0001:0000552b       convertToLittleEndian$fin$0 000000018000652b f   security.obj
 0001:0000555c       generateKeyBlob$fin$0      000000018000655c f   security.obj
 0001:0000557b       ?fin$0@?0??dllmain_crt_process_attach@@YAHQEAUHINSTANCE__@@QEAX@Z@4HA 000000018000657b f   MSVCRT:dll_dllmain.obj
 0001:00005592       ?fin$0@?0??dllmain_crt_process_detach@@YAH_N@Z@4HA 0000000180006592 f   MSVCRT:dll_dllmain.obj
 0001:000055ab       ?fin$1@?0??dllmain_crt_process_detach@@YAH_N@Z@4HA 00000001800065ab f   MSVCRT:dll_dllmain.obj
 0001:000055bf       ?filt$0@?0??dllmain_dispatch@@YAHQEAUHINSTANCE__@@KQEAX@Z@4HA 00000001800065bf f   MSVCRT:dll_dllmain.obj
 0001:000055f5       ?catch$0@?0???2@YAPEAX_KAEBUnothrow_t@std@@@Z@4HA 00000001800065f5 f   MSVCRT:new_scalar_nothrow.obj
 0001:00005602       __catch$??2@YAPEAX_KAEBUnothrow_t@std@@@Z$0 0000000180006602 f   MSVCRT:new_scalar_nothrow.obj
 0001:00005613       __scrt_is_nonwritable_in_current_image$filt$0 0000000180006613 f   MSVCRT:utility.obj
 0002:00000378       ?trace$initializer$@@3P6AXXZEA 0000000180007378     security.obj
 0002:00000a38       GS_ExceptionPointers       0000000180007a38     MSVCRT:gs_report.obj
 0002:000012c0       $unwind$fprintf            00000001800082c0     security.obj
 0002:000012cc       $unwind$printf             00000001800082cc     security.obj
 0002:000012d8       $unwind$snprintf           00000001800082d8     security.obj
 0002:000012e8       $unwind$?CallStaticObjectMethod@JNIEnv_@@QEAAPEAV_jobject@@PEAV_jclass@@PEAU_jmethodID@@ZZ 00000001800082e8     security.obj
 0002:000012e8       $unwind$?CallVoidMethod@JNIEnv_@@QEAAXPEAV_jobject@@PEAU_jmethodID@@ZZ 00000001800082e8     security.obj
 0002:000012e8       $unwind$?NewObject@JNIEnv_@@QEAAPEAV_jobject@@PEAV_jclass@@PEAU_jmethodID@@ZZ 00000001800082e8     security.obj
 0002:000012f0       $unwind$Java_sun_security_mscapi_CKeyStore_removeCngKey 00000001800082f0     security.obj
 0002:000012f0       $unwind$Java_sun_security_mscapi_CKey_cleanUp 00000001800082f0     security.obj
 0002:000012f0       $unwind$__raise_securityfailure 00000001800082f0     MSVCRT:gs_report.obj
 0002:000012f0       $unwind$??2@YAPEAX_K@Z     00000001800082f0     MSVCRT:new_scalar.obj
 0002:000012f0       $unwind$??_Gtype_info@@UEAAPEAXI@Z 00000001800082f0     MSVCRT:std_type_info_static.obj
 0002:000012f0       $unwind$??0bad_alloc@std@@QEAA@AEBV01@@Z 00000001800082f0     MSVCRT:throw_bad_alloc.obj
 0002:000012f0       $unwind$??0bad_array_new_length@std@@QEAA@AEBV01@@Z 00000001800082f0     MSVCRT:throw_bad_alloc.obj
 0002:000012f0       $unwind$??0exception@std@@QEAA@AEBV01@@Z 00000001800082f0     MSVCRT:throw_bad_alloc.obj
 0002:000012f0       $unwind$__scrt_initialize_onexit_tables 00000001800082f0     MSVCRT:utility.obj
 0002:000012f0       $unwind$__scrt_release_startup_lock 00000001800082f0     MSVCRT:utility.obj
 0002:000012f0       $unwind$__scrt_uninitialize_crt 00000001800082f0     MSVCRT:utility.obj
 0002:000012f8       $unwind$Java_sun_security_mscapi_CKey_getContainerName 00000001800082f8     security.obj
 0002:0000130c       $unwind$Java_sun_security_mscapi_CKey_getKeyType 000000018000830c     security.obj
 0002:00001320       $unwind$Java_sun_security_mscapi_CKeyStore_loadKeysOrCertificateChains 0000000180008320     security.obj
 0002:00001354       $unwind$Java_sun_security_mscapi_CKeyStore_loadKeysOrCertificateChains$fin$0 0000000180008354     security.obj
 0002:0000135c       $unwind$Java_sun_security_mscapi_CKeyStore_storeCertificate 000000018000835c     security.obj
 0002:0000138c       $unwind$Java_sun_security_mscapi_CKeyStore_destroyKeyContainer$fin$0 000000018000838c     security.obj
 0002:0000138c       $unwind$Java_sun_security_mscapi_CKeyStore_removeCertificate$fin$0 000000018000838c     security.obj
 0002:0000138c       $unwind$Java_sun_security_mscapi_CKeyStore_storeCertificate$fin$0 000000018000838c     security.obj
 0002:0000138c       $unwind$Java_sun_security_mscapi_CPublicKey_00024CRSAPublicKey_getExponent$fin$0 000000018000838c     security.obj
 0002:0000138c       $unwind$Java_sun_security_mscapi_CPublicKey_00024CRSAPublicKey_getModulus$fin$0 000000018000838c     security.obj
 0002:0000138c       $unwind$Java_sun_security_mscapi_CSignature_signHash$fin$0 000000018000838c     security.obj
 0002:0000138c       $unwind$Java_sun_security_mscapi_CSignature_verifySignedHash$fin$0 000000018000838c     security.obj
 0002:0000138c       $unwind$generateKeyBlob$fin$0 000000018000838c     security.obj
 0002:0000138c       $unwind$?filt$0@?0??dllmain_dispatch@@YAHQEAUHINSTANCE__@@KQEAX@Z@4HA 000000018000838c     MSVCRT:dll_dllmain.obj
 0002:00001394       $unwind$Java_sun_security_mscapi_CKeyStore_removeCertificate 0000000180008394     security.obj
 0002:000013c0       $unwind$Java_sun_security_mscapi_CKeyStore_destroyKeyContainer 00000001800083c0     security.obj
 0002:000013e4       $unwind$Java_sun_security_mscapi_CKeyStore_generateRSAPrivateKeyBlob 00000001800083e4     security.obj
 0002:000013e4       $unwind$Java_sun_security_mscapi_CSignature_00024RSA_generatePublicKeyBlob 00000001800083e4     security.obj
 0002:000013ec       $unwind$Java_sun_security_mscapi_CKeyStore_storePrivateKey 00000001800083ec     security.obj
 0002:0000141c       $unwind$Java_sun_security_mscapi_CKeyPairGenerator_00024RSA_generateCKeyPair$fin$0 000000018000841c     security.obj
 0002:0000141c       $unwind$Java_sun_security_mscapi_CKeyStore_storePrivateKey$fin$0 000000018000841c     security.obj
 0002:0000141c       $unwind$Java_sun_security_mscapi_CPublicKey_getPublicKeyBlob$fin$0 000000018000841c     security.obj
 0002:0000141c       $unwind$Java_sun_security_mscapi_CRSACipher_cngEncryptDecrypt$fin$0 000000018000841c     security.obj
 0002:0000141c       $unwind$Java_sun_security_mscapi_CRSACipher_encryptDecrypt$fin$0 000000018000841c     security.obj
 0002:0000141c       $unwind$Java_sun_security_mscapi_CSignature_importECPublicKey$fin$0 000000018000841c     security.obj
 0002:0000141c       $unwind$Java_sun_security_mscapi_CSignature_importPublicKey$fin$0 000000018000841c     security.obj
 0002:0000141c       $unwind$Java_sun_security_mscapi_CSignature_signCngHash$fin$0 000000018000841c     security.obj
 0002:0000141c       $unwind$Java_sun_security_mscapi_CSignature_verifyCngSignedHash$fin$0 000000018000841c     security.obj
 0002:00001424       $unwind$Java_sun_security_mscapi_PRNG_generateSeed 0000000180008424     security.obj
 0002:00001454       $unwind$Java_sun_security_mscapi_PRNG_generateSeed$fin$0 0000000180008454     security.obj
 0002:00001454       $unwind$convertToLittleEndian$fin$0 0000000180008454     security.obj
 0002:00001454       $unwind$?fin$0@?0??dllmain_crt_process_attach@@YAHQEAUHINSTANCE__@@QEAX@Z@4HA 0000000180008454     MSVCRT:dll_dllmain.obj
 0002:00001454       $unwind$?fin$0@?0??dllmain_crt_process_detach@@YAH_N@Z@4HA 0000000180008454     MSVCRT:dll_dllmain.obj
 0002:00001454       $unwind$?fin$1@?0??dllmain_crt_process_detach@@YAH_N@Z@4HA 0000000180008454     MSVCRT:dll_dllmain.obj
 0002:0000145c       $unwind$Java_sun_security_mscapi_PRNG_getContext 000000018000845c     security.obj
 0002:00001464       $unwind$??__Etrace@@YAXXZ  0000000180008464     security.obj
 0002:00001464       $unwind$Java_sun_security_mscapi_PRNG_releaseContext 0000000180008464     security.obj
 0002:00001464       $unwind$__scrt_initialize_default_local_stdio_options 0000000180008464     MSVCRT:default_local_stdio_options.obj
 0002:00001464       $unwind$?dllmain_crt_dispatch@@YAHQEAUHINSTANCE__@@KQEAX@Z 0000000180008464     MSVCRT:dll_dllmain.obj
 0002:00001464       $unwind$DllMain            0000000180008464     MSVCRT:dll_dllmain_stub.obj
 0002:00001464       $unwind$__GSHandlerCheck   0000000180008464     MSVCRT:gshandler.obj
 0002:00001464       $unwind$__scrt_acquire_startup_lock 0000000180008464     MSVCRT:utility.obj
 0002:00001464       $unwind$__scrt_dllmain_after_initialize_c 0000000180008464     MSVCRT:utility.obj
 0002:00001464       $unwind$__scrt_dllmain_before_initialize_c 0000000180008464     MSVCRT:utility.obj
 0002:00001464       $unwind$__scrt_dllmain_crt_thread_attach 0000000180008464     MSVCRT:utility.obj
 0002:00001464       $unwind$__scrt_dllmain_crt_thread_detach 0000000180008464     MSVCRT:utility.obj
 0002:00001464       $unwind$__scrt_dllmain_uninitialize_c 0000000180008464     MSVCRT:utility.obj
 0002:00001464       $unwind$__scrt_dllmain_uninitialize_critical 0000000180008464     MSVCRT:utility.obj
 0002:00001464       $unwind$__scrt_initialize_crt 0000000180008464     MSVCRT:utility.obj
 0002:0000146c       $unwind$Java_sun_security_mscapi_CRSACipher_encryptDecrypt 000000018000846c     security.obj
 0002:000014a0       $unwind$Java_sun_security_mscapi_CRSACipher_cngEncryptDecrypt 00000001800084a0     security.obj
 0002:000014d0       $unwind$Java_sun_security_mscapi_CKeyPairGenerator_00024RSA_generateCKeyPair 00000001800084d0     security.obj
 0002:00001500       $unwind$Java_sun_security_mscapi_CPublicKey_getPublicKeyBlob 0000000180008500     security.obj
 0002:00001530       $unwind$Java_sun_security_mscapi_CPublicKey_00024CRSAPublicKey_getExponent 0000000180008530     security.obj
 0002:0000155c       $unwind$Java_sun_security_mscapi_CPublicKey_00024CRSAPublicKey_getModulus 000000018000855c     security.obj
 0002:0000158c       $unwind$Java_sun_security_mscapi_CSignature_signCngHash 000000018000858c     security.obj
 0002:000015bc       $unwind$Java_sun_security_mscapi_CSignature_verifyCngSignedHash 00000001800085bc     security.obj
 0002:000015e8       $unwind$Java_sun_security_mscapi_CSignature_signHash 00000001800085e8     security.obj
 0002:0000161c       $unwind$Java_sun_security_mscapi_CSignature_verifySignedHash 000000018000861c     security.obj
 0002:00001650       $unwind$Java_sun_security_mscapi_CSignature_importPublicKey 0000000180008650     security.obj
 0002:0000167c       $unwind$Java_sun_security_mscapi_CSignature_importECPublicKey 000000018000867c     security.obj
 0002:000016ac       $unwind$dump               00000001800086ac     security.obj
 0002:000016c4       $unwind$ThrowExceptionWithMessage 00000001800086c4     security.obj
 0002:000016c4       $unwind$new[]              00000001800086c4     security.obj
 0002:000016c4       $unwind$_RTC_Initialize    00000001800086c4     MSVCRT:initsect.obj
 0002:000016c4       $unwind$_RTC_Terminate     00000001800086c4     MSVCRT:initsect.obj
 0002:000016c4       $unwind$??_Gbad_alloc@std@@UEAAPEAXI@Z 00000001800086c4     MSVCRT:throw_bad_alloc.obj
 0002:000016c4       $unwind$??_Gbad_array_new_length@std@@UEAAPEAXI@Z 00000001800086c4     MSVCRT:throw_bad_alloc.obj
 0002:000016c4       $unwind$??_Gexception@std@@UEAAPEAXI@Z 00000001800086c4     MSVCRT:throw_bad_alloc.obj
 0002:000016d0       $unwind$ThrowExceptionWithMessageAndErrcode 00000001800086d0     security.obj
 0002:000016e8       $unwind$ThrowException     00000001800086e8     security.obj
 0002:00001700       $unwind$MapHashAlgorithm   0000000180008700     security.obj
 0002:00001700       $unwind$MapHashIdentifier  0000000180008700     security.obj
 0002:00001700       $unwind$__scrt_dllmain_exception_filter 0000000180008700     MSVCRT:utility.obj
 0002:00001714       $unwind$GetCertificateChain 0000000180008714     security.obj
 0002:0000171c       $unwind$convertToLittleEndian 000000018000871c     security.obj
 0002:0000174c       $unwind$generateKeyBlob    000000018000874c     security.obj
 0002:0000177c       $unwind$__GSHandlerCheckCommon 000000018000877c     MSVCRT:gshandler.obj
 0002:00001784       $unwind$__GSHandlerCheck_SEH 0000000180008784     MSVCRT:gshandlerseh.obj
 0002:000017a0       $xdatasym                  00000001800087a0     MSVCRT:chkstk.obj
 0002:000017a8       $xdatasym                  00000001800087a8     MSVCRT:amdsecgs.obj
 0002:000017ac       $unwind$?dllmain_crt_process_attach@@YAHQEAUHINSTANCE__@@QEAX@Z 00000001800087ac     MSVCRT:dll_dllmain.obj
 0002:000017e8       $unwind$?dllmain_crt_process_detach@@YAH_N@Z 00000001800087e8     MSVCRT:dll_dllmain.obj
 0002:0000183c       $unwind$?dllmain_dispatch@@YAHQEAUHINSTANCE__@@KQEAX@Z 000000018000883c     MSVCRT:dll_dllmain.obj
 0002:00001864       $unwind$_DllMainCRTStartup 0000000180008864     MSVCRT:dll_dllmain.obj
 0002:00001874       $unwind$??2@YAPEAX_KAEBUnothrow_t@std@@@Z 0000000180008874     MSVCRT:new_scalar_nothrow.obj
 0002:00001884       $cppxdata$??2@YAPEAX_KAEBUnothrow_t@std@@@Z 0000000180008884     MSVCRT:new_scalar_nothrow.obj
 0002:00001891       $stateUnwindMap$??2@YAPEAX_KAEBUnothrow_t@std@@@Z 0000000180008891     MSVCRT:new_scalar_nothrow.obj
 0002:00001894       $tryMap$??2@YAPEAX_KAEBUnothrow_t@std@@@Z 0000000180008894     MSVCRT:new_scalar_nothrow.obj
 0002:0000189c       $handlerMap$??2@YAPEAX_KAEBUnothrow_t@std@@@Z 000000018000889c     MSVCRT:new_scalar_nothrow.obj
 0002:000018a4       $ip2state$??2@YAPEAX_KAEBUnothrow_t@std@@@Z 00000001800088a4     MSVCRT:new_scalar_nothrow.obj
 0002:000018a8       $unwind$?catch$0@?0???2@YAPEAX_KAEBUnothrow_t@std@@@Z@4HA 00000001800088a8     MSVCRT:new_scalar_nothrow.obj
 0002:000018b8       $cppxdata$?catch$0@?0???2@YAPEAX_KAEBUnothrow_t@std@@@Z@4HA 00000001800088b8     MSVCRT:new_scalar_nothrow.obj
 0002:000018c2       $stateUnwindMap$?catch$0@?0???2@YAPEAX_KAEBUnothrow_t@std@@@Z@4HA 00000001800088c2     MSVCRT:new_scalar_nothrow.obj
 0002:000018c4       $ip2state$?catch$0@?0???2@YAPEAX_KAEBUnothrow_t@std@@@Z@4HA 00000001800088c4     MSVCRT:new_scalar_nothrow.obj
 0002:000018c8       $unwind$__report_gsfailure 00000001800088c8     MSVCRT:gs_report.obj
 0002:000018d0       $unwind$capture_previous_context 00000001800088d0     MSVCRT:gs_report.obj
 0002:000018dc       $unwind$__security_init_cookie 00000001800088dc     MSVCRT:gs_support.obj
 0002:000018e8       $unwind$__scrt_is_nonwritable_in_current_image 00000001800088e8     MSVCRT:utility.obj
 0002:00001908       $unwind$__scrt_is_nonwritable_in_current_image$filt$0 0000000180008908     MSVCRT:utility.obj
 0002:00001910       $unwind$__scrt_fastfail    0000000180008910     MSVCRT:utility_desktop.obj
 0002:00001920       $unwind$__isa_available_init 0000000180008920     MSVCRT:cpu_disp.obj
 0002:00001938       $xdatasym                  0000000180008938     MSVCRT:guard_dispatch.obj
 0002:00001940       $xdatasym                  0000000180008940     MSVCRT:guard_xfg_dispatch.obj
 0002:00001944       $unwind$?__scrt_throw_std_bad_alloc@@YAXXZ 0000000180008944     MSVCRT:throw_bad_alloc.obj
 0002:00001944       $unwind$?__scrt_throw_std_bad_array_new_length@@YAXXZ 0000000180008944     MSVCRT:throw_bad_alloc.obj
 0002:00001a40       .edata                     0000000180008a40     sunmscapi.exp
 0002:00001a68       rgpv                       0000000180008a68     sunmscapi.exp
 0002:00001ad0       rgszName                   0000000180008ad0     sunmscapi.exp
 0002:00001b38       rgwOrd                     0000000180008b38     sunmscapi.exp
 0002:00001b6c       szName                     0000000180008b6c     sunmscapi.exp
 0002:00001b7a       $N00001                    0000000180008b7a     sunmscapi.exp
 0002:00001bbf       $N00002                    0000000180008bbf     sunmscapi.exp
 0002:00001bf6       $N00003                    0000000180008bf6     sunmscapi.exp
 0002:00001c33       $N00004                    0000000180008c33     sunmscapi.exp
 0002:00001c72       $N00005                    0000000180008c72     sunmscapi.exp
 0002:00001ca7       $N00006                    0000000180008ca7     sunmscapi.exp
 0002:00001cd7       $N00007                    0000000180008cd7     sunmscapi.exp
 0002:00001d0b       $N00008                    0000000180008d0b     sunmscapi.exp
 0002:00001d3e       $N00009                    0000000180008d3e     sunmscapi.exp
 0002:00001d64       $N00010                    0000000180008d64     sunmscapi.exp
 0002:00001d93       $N00011                    0000000180008d93     sunmscapi.exp
 0002:00001dbc       $N00012                    0000000180008dbc     sunmscapi.exp
 0002:00001dff       $N00013                    0000000180008dff     sunmscapi.exp
 0002:00001e41       $N00014                    0000000180008e41     sunmscapi.exp
 0002:00001e76       $N00015                    0000000180008e76     sunmscapi.exp
 0002:00001eac       $N00016                    0000000180008eac     sunmscapi.exp
 0002:00001edf       $N00017                    0000000180008edf     sunmscapi.exp
 0002:00001f22       $N00018                    0000000180008f22     sunmscapi.exp
 0002:00001f58       $N00019                    0000000180008f58     sunmscapi.exp
 0002:00001f8c       $N00020                    0000000180008f8c     sunmscapi.exp
 0002:00001fbc       $N00021                    0000000180008fbc     sunmscapi.exp
 0002:00001fe9       $N00022                    0000000180008fe9     sunmscapi.exp
 0002:00002021       $N00023                    0000000180009021     sunmscapi.exp
 0002:00002056       $N00024                    0000000180009056     sunmscapi.exp
 0002:00002081       $N00025                    0000000180009081     sunmscapi.exp
 0002:000020aa       $N00026                    00000001800090aa     sunmscapi.exp
 0002:0000266e       .idata$6                   000000018000966e     advapi32:ADVAPI32.dll
 0002:00002824       .idata$6                   0000000180009824     crypt32:CRYPT32.dll
 0002:0000290c       .idata$6                   000000018000990c     ncrypt:ncrypt.dll
 0002:00002aa0       .idata$6                   0000000180009aa0     kernel32:KERNEL32.dll
 0002:00002b68       .idata$6                   0000000180009b68     vcruntime:VCRUNTIME140.dll
 0002:00002b7a       .idata$6                   0000000180009b7a     vcruntime:VCRUNTIME140_1.dll
 0002:00002ce0       .idata$6                   0000000180009ce0     ucrt:api-ms-win-crt-stdio-l1-1-0.dll
 0002:00002d00       .idata$6                   0000000180009d00     ucrt:api-ms-win-crt-convert-l1-1-0.dll
 0002:00002d22       .idata$6                   0000000180009d22     ucrt:api-ms-win-crt-environment-l1-1-0.dll
 0002:00002d48       .idata$6                   0000000180009d48     ucrt:api-ms-win-crt-string-l1-1-0.dll
 0002:00002d6a       .idata$6                   0000000180009d6a     ucrt:api-ms-win-crt-runtime-l1-1-0.dll
 0002:00002d8c       .idata$6                   0000000180009d8c     ucrt:api-ms-win-crt-heap-l1-1-0.dll
 0003:00000130       ?__proc_attached@@3HA      000000018000a130     MSVCRT:dll_dllmain.obj
 0003:00000140       GS_ExceptionRecord         000000018000a140     MSVCRT:gs_report.obj
 0003:000001e0       GS_ContextRecord           000000018000a1e0     MSVCRT:gs_report.obj
 0003:000006d8       ?is_initialized_as_dll@@3_NA 000000018000a6d8     MSVCRT:utility.obj
 0003:000006d9       ?module_local_atexit_table_initialized@@3_NA 000000018000a6d9     MSVCRT:utility.obj
 0003:000006e0       ?module_local_atexit_table@@3U_onexit_table_t@@A 000000018000a6e0     MSVCRT:utility.obj
 0003:000006f8       ?module_local_at_quick_exit_table@@3U_onexit_table_t@@A 000000018000a6f8     MSVCRT:utility.obj
 0005:00000060       $R000000                   000000018000c060     sunmscapi.dll.res
